:0400000081313629EB
:1000080080310310003003180130F4002000111D66
:100018000E280F28C1280130AC070030AD3D003054
:10002800AE3D0030AF3D7508031D1B2886287808B3
:10003800031D1F2886287608F000F101F201F3015C
:1000480073082F02031D322872082E02031D32285E
:1000580071082D02031D322870082C020318352858
:10006800362838288D163A288D123A2800302F0263
:10007800031D482800302E02031D482800302D0299
:10008800031D482829302C02031C4B284C2886289D
:100098007608013EF000003003180130F1007108C5
:1000A800803AFF0080307F02031D5C2828307002F0
:1000B80003185F2860286E280130F0007008F607E2
:1000C80000302000AF000030AE000030AD0000303E
:1000D800AC008628200018100030AF000030AE00B9
:1000E8000030AD000030AC000310003003180130C0
:1000F800F6004130970096018D16111135293529E2
:100108008628862800302F02031D942800302E02EE
:10011800031D942800302D02031D942806302C025C
:10012800031C97289828BD28F508031D9C289D289E
:10013800BD287808031DA128AD28F5010314F50D85
:1001480018109801250092013E30910020001814E3
:10015800BD283008031DB128B3288D16B3280030F8
:10016800AF000030AE000030AD000030AC00BD285C
:10017800BD28970196011111C128111CC428C52852
:10018800C6281110911DC928CA2835292400141918
:10019800CE28CF281829141CD228D3283229110890
:1001A800F0007008F400082903100030031801302B
:1001B8002000B0000310003003180130F8008D1241
:1001C800322903100030031801302000B00003105A
:1001D800003003180130F8008D16322920008D16E2
:1001E800B0010314B00D0310003003180130F800FB
:1001F800322920008D16B0010314B00DF801031444
:10020800F80D3229322932297408113A0319D828ED
:10021800333A0319E528113A0319F228773A0319F2
:10022800FD28322932293229941E1B291C2922290A
:100238001108F0007008F40096123229770891002E
:1002480015162629141829292A2926292B290310A5
:10025800003003180130F7003229322920009111AB
:100268003529090088018231972A00342334303433
:100278002A34393438343734363435343434333432
:100288003234313403100030031801302000AB0041
:100298000310003003180130AA000030A900003014
:1002A800A8000030A7000030A6007F30A400240872
:1002B800210095058B0198308E0007302000A4009E
:1002C80024088E040F3021008D0020008D16240094
:1002D8000D148D140D158D15F0302000A400240880
:1002E80023008D05E230210099000F3098008E1709
:1002F8000E170C3023009B0090309D0024309E0088
:1003080000302000A9000030A8000030A70000300D
:10031800A60000302902031D9B2900302802031D76
:100328009B2900302702031D9B2964302602031CE9
:100338009E299F29A129BC29BC290130A607003084
:10034800A73D0030A83D0030A93D00302902031D1B
:10035800B72900302802031DB72900302702031DE2
:10036800B72964302602031CBA29BB29A129BC2954
:100378008231B52281310A30250093008B170B1783
:1003880021001115911520009111823180228131AF
:10039800413020009700D0290310003003180130A5
:1003A800AB0003302B02031CDA29DB29DD29D02915
:1003B800D0290130A4002B0AE229A435890BE129B0
:1003C8002408FF3AA50025088E05031000300318FD
:1003D8000130AA0004302A02031CF329F429F62963
:1003E800482A482A0130A4002A0AFB29A435890B87
:1003F800FA2924080D05031D022A032A3C2A413044
:100408001702031C082A092A3C2A3008031D0D2A52
:10041800142A8D120310003003180130F500142A35
:10042800823180228131200018140330A40024086E
:10043800A0002A088231622281313A3E20002B072F
:1004480081310A008231A5002508F7000330A40095
:100458002408A0002A088231622281313A3E200015
:100468002B0781310A0082318231A92281313C2A4D
:1004780001302000A4002408AA0704302A02031C23
:10048800462A472AF629482A0130A4002B0A4D2A71
:10049800A435890B4C2A2408A50025088E040130B0
:1004A800A4002408AB0703302B02031C5C2A5D2A36
:1004B800DD29D029D029D029813136292000A3006F
:1004C8000310003003180130A2006A2A231C6D2A89
:1004D8006E2A732A2008A1002108A207732A031094
:1004E800A00D0310A30CA308031D7B2A7C2A6A2AEB
:1004F8007D2A22087F2A0800200018103030980032
:10050800F4302500920024309100200097019601D4
:10051800111011110030AF000030AE000030AD00F6
:100528000030AC000800F501F601F701AC01AD019F
:10053800AE01AF018231BF228231F8008231BE2282
:100548008231B0002000813146292000A000AC2A69
:10055800111EAF2AB02AAC2AB12A200823009A001B
:1005680008002E3024009500E430920016109710F1
:080578001710080001340134E2
:00000001FF
